:1000000000308A001F2D00000A108A100A11820792
:1000100053347434613472347434213421340034F0
:100020000A108A100A11820756343D3425343234BE
:100030002E343234663420344C344D345434253428
:1000400031342E343234663400340A108A100A11E6
:10005000820741343D34253431342E343234663411
:1000600020344D3461347834253431342E343234F4
:10007000663400343C308400000803194C280630F4
:10008000F800F701F70B4228F80B41287B30F70006
:10009000F70B4828800B3F2800345308F039D5006F
:1000A00006080F395504D7008600D408031D5A28C6
:1000B00006155B2806110000861500000000861159
:1000C00000343B08D3000130D4004D203B0EBC006F
:1000D000F030BC053C08D3000130D4004D20023084
:1000E000BC003A2000340030831686000F308312A3
:1000F000BC003A203030D3000130D4004D20053010
:10010000BC003A203030D3000130D4004D20013003
:10011000BC003A203030D3000130D4004D200130F3
:10012000BC003A202030D3000130D4004D200130F3
:10013000BC003A202E30BB0061200830BB0061209B
:100140000D30BB0061200630BB0061200230BB00D7
:1001500061208A110A12392D0130BB0061200F3055
:10016000BC003A2000345108D300D4014D20510E78
:10017000D200F030D2055208D300D4014D205330C4
:10018000F700F70BC12800348E30F7003C08F80068
:100190003B08F900FA01F808031DD8287908F8008F
:1001A000F9010830F702F808031DD828F701E02804
:1001B0000310F81BDF28F90DF80DF703D828F81302
:1001C000000000343B0803195329C3003F080319FA
:1001D0005329C307031CED28F4287F30C302031CF6
:1001E000532903195329F8288130C30703185329C9
:1001F0004308F700F801F901FA013C08C700C717E6
:100200003D08C6003E08C5001830C300C401451CA7
:1002100021294208FA07031C1329F90A031D13298F
:10022000F80A0319C4174108F907031C1A29F80A28
:100230000319C4174008BD00BD173D08F80703188F
:10024000C417C40DF80CF90CFA0CC70CC60CC50C7D
:100250000310C30B06290130F70703185329F81BB5
:100260003829C70DFA0DF90DF80DF70303195329B5
:10027000C71F4929FA0A031D4929F90A031D4929FB
:10028000F80A031D4929F80CF90CFA0CF70A0319AE
:1002900053293C08C4004008C406C41F5129F8175C
:1002A0005729F8135729F701F801F901FA0100005D
:1002B00000343F0803191F2ACB00430803191F2AE3
:1002C000CB020318642969297F30CB0703181F2A42
:1002D0006F298130CB02031C1F2A03191F2A4B08E8
:1002E000F700F801F901FA01CA014008C900C9176D
:1002F0004108C8004208C7001930CB004608C702B1
:10030000031892290130C80203189229C902031860
:100310009229CA0203189229CA0AC90AC80A4608B9
:10032000C707C4294508C8020318AD290130C9020E
:100330000318AD29CA020318AD29CA0AC90A45081B
:10034000C8074608C707031CC429C80A031DC429D7
:10035000C90A031DC429CA0AC42944088038C9022D
:100360000318C3290130CA020318C329CA0A440862
:100370008038C9074508C807031CA129C90A031DFD
:10038000A129CA0AA1297A14CB0BC729D2290310A3
:10039000C70DC80DC90DCA0D0310FA0DF90DF80DE2
:1003A000CC0D7E294C1CDA290310F80CF90CFA0C40
:1003B000CC0CDD29F70303191F2ACC1B062A0310D6
:1003C000C70DC80DC90DCA0D4608C7020318F2298A
:1003D0000130C8020318F229C9020318F229CA021F
:1003E000031C152A4508C8020318FD290130C9025B
:1003F0000318FD29CA02031C152A44088038C902C3
:100400000318062A0130CA02031C152AFA0A031D22
:10041000152AF90A031D152AF80A031D152AF70AD9
:1004200003191F2AF80CF90CFA0C4008CB004408F9
:10043000CB06CB1F1D2AF817232AF813232AF7010E
:10044000F801F901FA010000003480300318C806F1
:10045000CD01CE014408CC004808CC06430803195E
:10046000132BCB00F700470803191C2BCB020319F1
:10047000B92A03183C2A782A4808D100D11749081C
:10048000D0004A08CF00CE010310D10CD00CCF0C05
:10049000CE0CCB0B432ACC1F502A4D14302B4D10C1
:1004A0004B104D1646308400462B4D12CC1B622A51
:1004B0004B1C6D2AD10CD00CCF0CCE0CF70A0319B3
:1004C0002B2B6D2AD11B702A0310CE0DCF0DD00D12
:1004D000D10DF70303192B2B622A4D17D82A4D1380
:1004E0004408CC00CC1F762AD117242BD113242BFF
:1004F0004708CB00F7004308CB024408D100D117CE
:100500004508D0004608CF00CE010310D10CD00C16
:10051000CF0CCE0CCB0B842ACC1F912ACD14302BC0
:10052000CD104B10CD164A308400462BCD12CC1B7B
:10053000A32A4B1CAE2AD10CD00CCF0CCE0CF70A40
:1005400003192B2BAE2AD11BB12A0310CE0DCF0DD0
:10055000D00DD10DF70303192B2BA32ACD17D82AC1
:10056000CD134808CC00CC1FB72AD117242BD113A8
:10057000242B4808D100D1174908D0004A08CF00E1
:10058000CC1FC62AD1134D15302B4D11CE014B1067
:1005900046308400462BCC1BEE2A4408CC004B1C72
:1005A000D82AD10CD00CCF0CCE0CF70A03192B2B68
:1005B000CE1FE92ACF0A031DE92AD00A031DE92A22
:1005C000D10A031DE92AD10CD00CCF0CF70A03196C
:1005D0002B2B4D1B6F2ACD1BB02A0D2B8030D10643
:1005E000D11FF62A302B4808CC00032B4408CC003E
:1005F000D108031D032BD008031D032BCF08031DB7
:10060000032BF701242BD11B0D2B0310CE0DCF0D87
:10061000D00DD10DF70B032B2B2BCC1F112BD1178A
:10062000242BD113242B4708F7004808D100490890
:10063000D0004A08CF00242B4308F7004408D1001B
:100640004508D0004608CF005108F8005008F900CE
:100650004F08FA00652BF701F801F901FA01652B43
:10066000CE01CF09D009D109CE09CE0A031D3F2BF7
:10067000CF0A031D3F2BD00A031D3F2BD10A4D1873
:100680004F2ACD18902A4D19C52AF32A0008CF0702
:10069000031C502BD00A031D502BD10A03194B14F5
:1006A00084030008D007031C582BD10A03194B14EC
:1006B00084030008801B5D2B803AD10703184B147C
:1006C0004D1A552ACD1A962ACB2A00000034040868
:1006D000C500C601BD1F6F2B2D30D100B320BD1743
:1006E0003C080319132C7F303C02031CCE2BBC00AA
:1006F000CB010430CC000310BF0DBE0DBD0DC60DE7
:10070000CC0B7B2B04303C0203188E2B03303C02B5
:10071000031D082C0A304602031C082C0330BC02BF
:10072000CB0AAF240310BF0DBE0DBD0DC60D98241E
:100730000230CC000310C60CBD0CBE0CBF0CCC0BA1
:100740009A2BAF240430CC000310C70CC80CC90C82
:10075000CA0CCC0BA42B9824AF244908CA00480823
:10076000C9004708C800C7019824AF244808CA0038
:100770004708C900C701C8019824C619822BBC08C4
:10078000031DC72BBF0ABE0ABD0AC60A082C0310E8
:10079000BF0DBE0DBD0DC60DBC03822BBC09BC0A2E
:1007A0007F30BC07CB010430CC000310BF0DBE0D61
:1007B000BD0DC60DCC0BD52B0430BC0705303C025B
:1007C000031C152CAF240310BF0DBE0DBD0DC60DAF
:1007D0000310BF0DBE0DBD0DC60D98240310BF0D37
:1007E000BE0DBD0DC60DCB0A0330CC000310C60CE8
:1007F000BD0CBE0CBF0CCC0BF62B0330BC02461E4E
:10080000DE2B0310C60CBD0CBE0CBF0CBC03DE2BD4
:10081000BC09BC0A0330BC074B08C1004B08C3002D
:10082000450AC3073F2C450ACB003030D100B32026
:10083000C508031D1C2C962C2E30D100B3204B086C
:10084000C400C40345084402031C282C4508C40006
:10085000C408031D2C2C322C30303030D100B32092
:10086000C40B2C2C4B08CC00450ACC020318B82C26
:10087000BC03450AC3004B08C3024308C100460835
:10088000C0003C080319492CC2000310C00CC20B65
:10089000452C43080319962C30304007D100B32073
:1008A0004108031D5A2CC508031D572C962C2E30C9
:1008B000D100B320C103C3030319962C3C080319CC
:1008C000662CC2000310C00DC20B622C4008C60289
:1008D0004608C7003D08C8003E08C9003F08CA00D6
:1008E0000310BF0DBE0DBD0DC60D0310BF0DBE0D17
:1008F000BD0DC60D4A08BF07031C832CBE0F832CF9
:10090000BD0F832CC60A4908BE07031C8A2CBD0FE5
:100910008A2CC60A4808BD070318C60A4708C60736
:100920000310BF0DBE0DBD0DC60D3F2C0000B82C31
:100930004A08BF07031CA12CBE0FA12CBD0FA12C80
:10094000C60A4908BE07031CA82CBD0FA82CC60A5E
:100950004808BD070318C60A4708C60700344608FA
:10096000C7003D08C8003E08C9003F08CA0000345F
:10097000000000343C08C3004008C306C31FC52C58
:1009800003110310BC1B0314F82C3C08C3003F08E0
:10099000C4003B08C4020319D32CC31FF82C03085E
:1009A000013A8300F82C4008C4003C08C402031933
:1009B000DF2CC31FF82C0308013A8300F82C4108F0
:1009C000C4003D08C4020319EB2CC31FF82C030814
:1009D000013A8300F82C4208C4003E08C4020319FF
:1009E000F72CC31FF82C0308013A8300F82C0310DE
:1009F0008A110A126B2F8E30F7003F08F702400869
:100A0000F9004108F800F917F708031D082D142D07
:100A10000310F908031D102DF808031D102D142DC7
:100A2000F90CF80CF70B082DC01F1B2DF809F9095C
:100A3000F80A0319F90A00008A110A129E2F84018C
:100A40001F308305073083169F0083128230831680
:100A50009F0083121F08383981389F0000308316A9
:100A60008600831286010030831687008312870177
:100A70007328AC20BB013B080420BB0AF700D1005F
:100A8000B32007303B02031D3B2D0430BB00FA307E
:100A9000BC003A20BB0B472DAC201830F8001F08D3
:100AA000C73978049F005330F700F70B552D1F15F9
:100AB0001F19582D1E08FA0083161E088312BB004A
:100AC0007A08BC00C4207A08B0007908AF00780822
:100AD000AE007708AD003008BE002F08BD002E081C
:100AE000BC002D08BB00C201C1017030C0008230C3
:100AF000BF00E2207708BB007808BC007908BD0081
:100B00007A08BE00C2003D08C1003C08C0003B0896
:100B1000BF00C601C501C4018930C30059217A084C
:100B2000B0007908AF007808AE007708AD00083053
:100B3000F8001F08C73978049F005330F700F70BFF
:100B40009F2D1F151F19A22D1E08FA0083161E08BF
:100B50008312BB007A08BC00C4207A08A40079087C
:100B6000A3007808A2007708A1009A30BE0099304F
:100B7000BD002930BC008130BB002408C20023081E
:100B8000C1002208C0002108BF00E2207708BB0096
:100B90007808BC007908BD007A08BE00C2003D0894
:100BA000C1003C08C0003B08BF00C601C501C4012C
:100BB0008930C30059217708BF007808C000790840
:100BC000C1007A08C20003144208C6004108C500EB
:100BD0004008C4003F08C3008F30CA00C230C900BB
:100BE0007530C8007B30C70025227A08A400790838
:100BF000A3007808A2007708A1001030F8001F08B1
:100C0000C73978049F005330F700F70B052E1F15E6
:100C10001F19082E1E08FA0083161E088312BB0037
:100C20007A08BC00C4207A08A8007908A7007808D0
:100C3000A6007708A5003330BE003330BD00133066
:100C4000BC008130BB002808C2002708C10026086C
:100C5000C0002508BF00E2207708BB007808BC0070
:100C60007908BD007A08BE00C2003D08C1003C08FA
:100C7000C0003B08BF00C601C501C4018930C300E4
:100C800059217708BF007808C0007908C1007A08A8
:100C9000C20003144208C6004108C5004008C40051
:100CA0003F08C300AE30CA004730C9002130C80039
:100CB0007F30C70025227A08A8007908A7007808A5
:100CC000A6007708A5000030F8001F08C73978048F
:100CD0009F005330F700F70B6B2E1F151F196E2E58
:100CE0001E08FA0083161E088312BB007A08BC0097
:100CF000C4207A08AC007908AB007808AA0077080D
:100D0000A9002C08BE002B08BD002A08BC00290839
:100D1000BB00C201C1012030C0008130BF00E22011
:100D20007708BB007808BC007908BD007A08BE00CF
:100D3000C2003D08C1003C08C0003B08BF00C6011E
:100D4000C501C4018930C30059217A08AC00790873
:100D5000AB007808AA007708A9002030F8001F0827
:100D6000C73978049F005330F700F70BB52E1F15D5
:100D70001F19B82E1E08FA0083161E088312BB0026
:100D80007A08BC00C4207A08B8007908B70078084F
:100D9000B6007708B5003808BE003708BD00360831
:100DA000BC003508BB00C201C1014830C00085301D
:100DB000BF00E2207A08B8007908B7007808B600CA
:100DC0007708B500AC205630D100B3203D30D100BB
:100DD000B320023084003008BF002F08BE002E0868
:100DE000BD002D08BC0067230730BB003B08102066
:100DF000BB0AF700D100B3200B303B02031DF62ED7
:100E0000023084002C08BF002B08BE002A08BD0059
:100E10002908BC006723C030BB0061204130D100ED
:100E2000B3203D30D100B320023084002408BF003D
:100E30002308BE002208BD002108BC00672307303C
:100E4000BB003B082520BB0AF700D100B3200B30C4
:100E50003B02031D212F023084002808BF00270811
:100E6000BE002608BD002508BC0067230314C60188
:100E7000C5017030C4008230C3003008CA002F089A
:100E8000C9002E08C8002D08C7002522C201C101D3
:100E90002030C0008230BF007A08C6007908C50043
:100EA0007808C4007708C30059217A08B40079088B
:100EB000B3007808B2007708B100BE01BD01BC01E3
:100EC0008030BB003408C2003308C1003208C000C3
:100ED0003108BF00BA2C03186E2F712F0F30B900E4
:100EE000A02F3408BE003308BD003208BC00310812
:100EF000BB00C201C1017030C0008230BF00E220DF
:100F00007708BB007808BC007908BD007A08BE00ED
:100F1000C2003D08C1003C08C0003B08BF00C6013C
:100F2000C501C4018030C30059217A08C200790884
:100F3000C1007808C0007708BF00FB2C7808B90012
:100F400039088700BA080319A82F8717BA01AB2FF1
:100F500087130130BA000230BB00FA30BC003A20DF
:080F6000BB0BAD2F4D2D63000A
:02400E00723FFF
:00000001FF
